:020000040002F8
:1060000000D10020C1630200C9630200CB6302001B
:10601000CD630200CF630200D163020000000000E4
:10602000000000000000000000000000D363020038
:10603000D563020000000000D7630200D9630200AC
:1060400041660200DB630200756802000967020016
:10605000DB630200DB6302009D650200DB6302007C
:10606000DB630200DB630200E5670200DB63020022
:10607000DB630200DB630200DB630200DB63020020
:10608000DB63020099660200DB630200DB6302004F
:10609000DB630200DB6302005D670200DB6302007A
:1060A000DB630200DB630200DB630200DB630200F0
:1060B000DB630200DB630200000000000000000060
:1060C000DB630200DB630200DB630200DB630200D0
:1060D000DB630200DB630200DB6302000000000000
:1060E00000000000000000000000000000000000B0
:1060F00000000000000000000000000000000000A0
:10610000000000000000000000000000000000008F
:10611000000000000000000000000000000000007F
:10612000000000000000000000000000000000006F
:10613000000000000000000000000000000000005F
:10614000000000000000000000000000000000004F
:10615000000000000000000000000000000000003F
:10616000000000000000000000000000000000002F
:10617000000000000000000000000000000000001F
:10618000000000000000000000000000000000000F
:1061900000000000000000000000000000000000FF
:1061A00000000000000000000000000000000000EF
:1061B00000000000000000000000000000000000DF
:1061C00000000000000000000000000000000000CF
:1061D00000000000000000000000000000000000BF
:1061E00000000000000000000000000000000000AF
:1061F000000000000000000000000000000000009F
:10620000DFF80CD000F08CF900480047D98A020072
:1062100000D1002030B450E8012F93B2C489234448
:106220008489A34228BF1B1B0489A34202BFBFF37A
:106230002F8F002007E0C3EA020340E80134002C5E
:10624000E9D14FF001000A6030BC704750E8012FDF
:10625000C2EA024240E801210029F7D1704730B478
:1062600050E8022F1FFAA2F3C488A34202BFBFF373
:106270002F8F00200DE0C48923448489A34228BFC6
:106280001B1BC2EA034340E80234002CE8D14FF064
:1062900001000A6030BC704750E8022FC2EA224277
:1062A00040E802210029F7D17047034653E8022F46
:1062B000D988B2EB324F4FF0000017BF92B241EADB
:1062C000014142EA014104E05A68B2EB324F08BF93
:1062D000012043E80212002AE8D1704730B4044696
:1062E00054E8000F0D4644E80053002BF8D1156028
:1062F00030BC704730B4044654E8000F40EA010552
:1063000044E80053002BF7D1156030BC704730B41F
:10631000044654E8000F00EA010544E80053002B4E
:10632000F7D1156030BC704730B4044654E8000F14
:1063300080EA010544E80053002BF7D1156030BC1A
:10634000704730B4044654E8000F00EB010544E800
:106350000053002BF7D1156030BC704730B40446B1
:1063600054E8000FA0EB010544E80053002BF7D1DF
:10637000156030BC704770B404464FF0000054E81C
:10638000006F0D68AE4207BF44E80023012044E8D7
:1063900000630E60002B1CBF0020F0E770BC70474C
:1063A00030B4044654E8000F88422CBF451A054615
:1063B00044E80053002BF5D1156030BC7047000055
:1063C0000648804706480047FEE7FEE7FEE7FEE78F
:1063D000FEE7FEE7FEE7FEE7FEE7FEE76167020095
:1063E000016202002DE9F05F0546002092469B46BF
:1063F00088460646814640241BE0284641464746DB
:10640000224600F07DF853465A46C01A914110D3F7
:1064100011461846224600F016F82D1A67EB0108BF
:106420004F4622460120002100F00DF817EB00092D
:106430004E41201EA4F10104DFDC484631462A46C5
:106440004346BDE8F09F202A04DB203A00FA02F11F
:10645000002070479140C2F1200320FA03F3194352
:1064600090407047004870470CB6020040EA0103B4
:106470009B0703D009E008C9121F08C0042AFAD2FA
:1064800003E011F8013B00F8013B521EF9D27047BE
:10649000D2B201E000F8012B491EFBD27047002266
:1064A000F6E710B513460A4604461946FFF7F0FF13
:1064B000204610BD421C10F8011B0029FBD1801A98
:1064C0007047034611F8012B00F8012B002AF9D17F
:1064D0001846704730B50B460146002020220124A3
:1064E00009E021FA02F59D4205D303FA02F5491BA2
:1064F00004FA02F52844151EA2F10102F1DC30BDB8
:10650000202A04DB203A21FA02F00021704721FA08
:1065100002F3D040C2F1200291400843194670476F
:10652000064C074D06E0E06840F0010394E80700E0
:1065300098471034AC42F6D3FFF766FE88BD0200E0
:10654000A8BD020070B58C1810F8015B15F00703A8
:1065500001D110F8013B2A1106D110F8012B03E0FC
:1065600010F8016B01F8016B5B1EF9D12B0705D404
:106570000023521E0DD401F8013BFAE710F8013B4D
:10658000CB1A921C03E013F8015B01F8015B521E69
:10659000F9D5A142D8D3002070BD00002DE9F84301
:1065A0000025DFF894804FF4807601242F46009573
:1065B000304602F0D7FF38B1D8F80403204203D0A8
:1065C000304602F0C5FF2543361D64007F1CB6B27D
:1065D000082FEDD34FF4BE74204602F0C3FF48B13C
:1065E000204602F0B5FF45F000456A460121002033
:1065F00002F062FF15F0FF0F16D0012600242E4294
:106600000ED008EB8401D1F81005D1F81015C0F3B5
:1066100004200A4AC1F3014152F8242002B19047F4
:106620007600641C082CEAD3002D02DA684604F0D8
:1066300063F9BDE8F88300000060004028A700204F
:1066400070B54FF48076304602F0AAFD114CB505C6
:1066500060B1304602F0ABFD0120C5F80803607957
:1066600020B9012060712168002088474FF48276AC
:10667000304602F095FD00280AD0304602F097FD22
:106680000220C5F808032168BDE8704001200847D2
:1066900070BD0000502B002002490248091F096804
:1066A00000680847BC2B002000F0EAB870B50E4621
:1066B000144900EB400001EBC0051446E86A1835A8
:1066C00020B101280FD0022805D113E0284600F0A0
:1066D0000BF9A04201D2002411E02246314628469F
:1066E00000F03AF90BE0284600F0FEF8A042F4D2A0
:1066F0000446F2E73146284600F001F904462046F8
:1067000070BD000074AE0020F8B51248124E044669
:106710004FF48C7103F0C9FC00281AD00025C4F88E
:106720001851D4F818010090F07F3446FF2806D0A5
:10673000A17F11B102F0D6FE01E002F0E9FE65771B
:106740002572D4E9002101B004F10800BDE8F04051
:106750001047F8BD00300040D4A7002003F01EBC55
:106760001B4800B5016841F470010160BFF34F8F11
:10677000BFF36F8F4FF01022D2F80002002803DB26
:10678000D2F8040200281FDA012003F03DFF152192
:10679000C2F800120F480368002BFCD0C2F80412A4
:1067A00001680029FCD0002003F02EFFBFF34F8FBB
:1067B00007487C380168084A01F4E0611143016030
:1067C000BFF34F8F00BFFDE705490448086000BDD7
:1067D00088ED00E000E401400400FA050090D003D9
:1067E000282C00202DE9FC411D48D0F8401100293B
:1067F00034D0D0F80413C90330D50023C0F8403199
:1068000004F002FA174800BFD0F804110029FBD0A9
:10681000C0F80431144CA069010402D56FF30F00D5
:10682000A0610246C0F3851060F39F120FA1684675
:1068300000F0B4F86846FFF73DFE62886D461146E9
:106840000B4E131803E08F1AEF5D7754491C8B42EF
:10685000F9DC10446080A068401CA060BDE8FC81A9
:1068600000A0004000700040D82A00200A256400E3
:10687000502C00200148006800470000582B0020E1
:1068800010B5124C02202061606111A0A06104F1DA
:106890007800E0614FF4007020620020A062606226
:1068A0000BA1A164E06204F51E71E1641021A065F2
:1068B000C4E91410E06509A1E01DFFF702FE08A17C
:1068C0002046FFF7FEFD2020A07110BD74AE002011
:1068D0005465726D696E616C000000005254540082
:1068E00053454747455200000269C1688A4203D8B0
:1068F0008068401A104400E0501A401E70472DE98D
:10690000F047C4681746894606464FF000083069CC
:10691000A04201D9051B02E0B168201A0D1AB06827
:106920006D1E001BA84200D80546BD4200D33D465F
:1069300070682A4620444946FFF798FDB0687F1BDF
:106940002C44A844A944A04200D10024F460002FA4
:10695000DDD14046BDE8F0872DE9F0410446884688
:10696000D4E90207C51BE168606816460844B542D1
:1069700006D94146FFF77AFDB819E060BDE8F0811D
:106980002A464146FFF772FD761B08EB05013246A9
:106990006068FFF76BFDE660F0E700000FB4084B9E
:1069A00010B504A902AA039800F02EF8044602A923
:1069B000002000F0D3F8204610BC5DF814FB000066
:1069C0005D6B020002E008C8121F08C1002AFAD15C
:1069D00070477047002001E001C1121F002AFBD15F
:1069E000704700000121202803DA8140054801405A
:1069F00003E0402802DA2038814009B101207047C5
:106A000000207047FC06FFBD2DE9FF4F89B09B4673
:106A10000446002506E025280BD05A460B999047DE
:106A2000641C6D1C20780028F5D10DB02846BDE807
:106A3000F08F0027B8460122474900E0074314F8C9
:106A4000013F203B02FA03F00842F7D120782E28BC
:106A500019D114F8010F47F004072A280ED06FF05F
:106A60002F022078A0F1300109290CD808EB880109
:106A700002EB410100EB0108641CF2E70A98641C78
:106A800050F8048B0A9020780028CED0642808D0D3
:106A9000692806D075281ED05A460B9990476D1C60
:106AA00058E00A994FF00A0901C90A91002802DA50
:106AB00040422D2102E0390504D52B218DF820100C
:106AC000012103E0F90704D02021F7E78A4608AE48
:106AD0000DE00021FAE70A994FF00A0901C90A916D
:106AE000F7E74946FFF7F6FC303106F8011D0028AC
:106AF000F7D1ADEB060000F12009780701D44FF083
:106B00000108C84502DDA8EB090000E0002080462E
:106B1000002706E008A85A46C05D0B9990476D1CF7
:106B20007F1C5745F6DB04E030205A460B9990470E
:106B30006D1CB8F10001A8F10108F5DC05E016F8BC
:106B4000010B5A460B9990476D1CB9F10001A9F150
:106B50000109F4DC641C65E7092801000A68531C7C
:106B60000B601070704790F82400012801D01F209E
:106B70007047EE20704710B501220221002000F07E
:106B8000DBFF08B1072810D107220221012000F005
:106B9000D3FF08B1072808D100210A22084600F0D7
:106BA000CBFF08B1072800D1002010BD70B500242C
:106BB000064D06E06868012110F8340003F004FB7C
:106BC000641C28788442F5D3002070BD602B00201F
:106BD000F8B516460C4605460A2A01D20720F8BD2C
:106BE00003F0ECFB18B903F0AFFB0028F7D1134F0B
:106BF000102113487D603C70BE60FFF750FC002000
:106C0000C7E904000F4E0DE005EBC40031680091A8
:106C100081788DF8011000780B4A694603F024FB57
:106C20000028DCD1641EE4B2EED2BDE8F84005488D
:106C30000021064A001D00F089B80000602B0020EA
:106C400018A8002050B302007D8802001D840200B5
:106C5000074910B5496801EBC004207803F06AFBCE
:106C60006178012901D0012100E00021484010BDD8
:106C7000602B002072B602F0F9FE00BF02F042FD68
:106C80000028FBD111481249401AC408012000EB2A
:106C9000044010A102F052FE11480068C00700D065
:106CA00000BE022000EB04400EA102F047FEBFF33D
:106CB0004F8F0B48E43801680E4A01F4E06111433C
:106CC0000160BFF34F8F00BFFDE7000020BE020050
:106CD000B8BD0200466174616C206572726F72000B
:106CE000F0ED00E053797374656D2072657365741F
:106CF000000000000400FA050EB500210091CDE966
:106D000001106A4644F20100FFF7B4FF0EBD10B552
:106D10008268C368934203D001F06AFD002010BD71
:106D2000052010BD10B58268C3689A1A83889A42FC
:106D300003D801F067FD002010BD042010BD000045
:106D4000014801F0D2BB0000802B00203AB100685E
:106D50000129426100D00021016100207047072015
:106D60007047000038B51148082358224168009147
:106D70000F49006802F013F8002815D10D4A694642
:106D80000D4801F0B7FB04000ED101210A4801F0C3
:106D90002CFC0123094A1946074801F07EFB0649ED
:106DA000012008390870204638BD000058B30200A1
:106DB00038A8002091AA0200802B0020FFFF7F004E
:106DC00070B50446007F0D4608B1002070BDA26179
:106DD00001F03AFD401941F10001C4E902012069C6
:106DE00000B125612146BDE87040002004F034B9AF
:106DF000014600200877012004F02EB910B50146A5
:106E00001048FFF78FFF040019D10F480F4A01788F
:106E1000515C19B1001D03F09DFB02E00C3003F042
:106E200033FB60B9084907480839FFF770FF30B9EC
:106E3000054901220839044802F0FCF904462046BD
:106E400010BD0000A0A80020A42B0020442B00208F
:106E500030B5EFF3108172B60D4A9468012324B166
:106E60000370002900D162B630BD93604FF0E0237B
:106E7000D3F88051074C25401560C3F88041D3F802
:106E8000844154605A17C3F8842100220270E8E755
:106E9000B0A80020FC06FFBD0B498A68002A11D06B
:106EA00000280FD1EFF3108072B60B684FF0E0228C
:106EB000C2F800314B68C2F8043100228A60002811
:106EC00000D162B670470000B0A8002070B5150070
:106ED000044609D00020286034B1206820B1A07990
:106EE000800703D0072070BD0E2070BD084600F05B
:106EF000D1FAC0B2142804D02179814203D80420E9
:106F000070BD052070BDE288216800FB021028607A
:106F1000002070BD2DE9FC47002517880646158026
:106F200090F82D001446894630B13A46214648462D
:106F300000F0C4FA051E09D1B0784FF00C0A18B35E
:106F40002088C846001DB84202D95046BDE8FC87DB
:106F5000684679DF0028F9D12088032108F800105D
:106F600020881921401C80B2208008F80010208859
:106F7000401C80B2208000EB0801BDF8000004F046
:106F8000A3F8218808442080F0780222C8B1218823
:106F900096F9033001F1030C4846BC45D5D842545C
:106FA00021884FF0010C491C89B2218000F801C0F2
:106FB0002188491C89B2218009F801302088401CB1
:106FC00020807068B8B1218890F9003001F1030C7D
:106FD0004846BC45B9D8425421880A22491C89B286
:106FE000218042542188491C89B2218009F801304E
:106FF0002088401C2080308950B1CDE900474B46A5
:107000000622022106F1080004F0ECF8051E9DD1CD
:10701000308A50B1CDE900474B460722032106F1E3
:10702000100004F0DFF8051E90D1308B50B1CDE98F
:1070300000474B461522142106F1180004F0D2F83F
:10704000051E83D1306A30B13B462246494601F0E5
:107050001CF9051EDBD1706A30B13B462246494619
:1070600001F0C0FD051ED2D196F82C0038B13B4688
:1070700022464946304603F065FE051EC7D13078EA
:1070800038B13B4622464946304601F035FE051EE2
:10709000BDD128465AE718B504460020ADF80000D7
:1070A00013466A46204600F006F8002802D0BDF8D4
:1070B0000000204418BD70B5E0B1DAB1002402E050
:1070C000045D2C44A4B2651C8D4206D21688A642EB
:1070D000F6D8061976789E42F2D18C420AD2A31CC9
:1070E000005D9BB200B1401E0004000C02D01C18D1
:1070F0008C4201D9002070BD138070BD80F8301023
:1071000070472DE9F0410D00044606D02CB195F8EA
:107110007A000026012803D006E00E20BDE8F081A9
:1071200095F89800012829D0D5F8A000042825D08A
:10713000D5F89C00042821D04FF00108A6702C221D
:1071400005F17801201DFFF791F984F83060D5F83A
:10715000A4006063D5F8A800A0634FF6FF70A4F800
:10716000240404F58260C4F82004C4F82664A4F85A
:107170002A6484F82C64207810B104E00720CDE75D
:10718000FF2084F8540004F155072046C4F8107419
:10719000FFF7E9FCA4F8140404F214423946284627
:1071A000FFF7B8FE0028B9D104F23120C4F8180462
:1071B0002046FFF7D8FCA4F81C0404F21C4205F199
:1071C0003C00D4F81814FFF7A5FE0028A6D184F8D7
:1071D0005180208BA4F8480084F83C80266484F811
:1071E0005060606900216064454604F13C02781EED
:1071F00072DF002892D1257090E710B50288102A1E
:107200001BD0112A20D0262A1DD1007A0C46012835
:1072100001D0022817D1A0780521401CB0FBF1F263
:1072200001FB1201204600F01DF800280BD0A16BD5
:10723000002908D0BDE810400847C27B012A02D1CE
:107240008088A1F8240410BD0C46002184F82E1477
:107250008088B4F824148842F5D120790028F2D12E
:107260000121DFE72DE9F05F044600780F4698B171
:10727000A7700025C4F82654A4F82A5484F82C5486
:10728000A079012608B1012F09D0E07980B1012F42
:1072900005D0022F03D00BE00820BDE8F09F616B02
:1072A00021B184F82D640820884701E084F82D542A
:1072B00004F2274100200A5C0AB1304603E0401C7A
:1072C0000628F8D300204FF002084FF0030B012FDF
:1072D00006D0022F0CD0032F0FD0042F15D110E0B1
:1072E000A17929B194F8241011B908B130460DE004
:1072F000E17911B108B1404608E0207A08B158465A
:1073000004E0607A08B1042000E02846A070616BB8
:1073100041B1032801D0042804D1607910B194F858
:107320002E0498B184F82F5404F13C00182107462C
:10733000FFF7B5F884F83C6004F12C0003F0ACFAD8
:1073400058B194F82C0084F8510008E084F83054C7
:1073500084F82F6407208847E6E784F8516094F8A2
:10736000240058B104F1280003F096FA20B194F8F3
:10737000280084F8520001E084F8526084F85050EC
:10738000A27804F2264104F582694FF0060A052A24
:1073900064D2DFE802F07C030F22420084F83160FF
:1073A000C4F82054C4E9101584F83C808020A4F867
:1073B000480055E084F8318094F82420384612B112
:1073C0000722027001E080F800B0228A8281C4F8AE
:1073D00020544160E168B96042E06069B860208B88
:1073E000B88194F824003D460028204602D084F855
:1073F0003CA001E084F83C6003F0C6FE50B185F883
:1074000014800421204601F00BFA38BB052184F8D2
:10741000311021E084F831B01EE0E069B860208CC2
:10742000B88194F824003D460028204602D084F814
:107430003CA001E084F83C6003F0A6FE48B185F86A
:1074400014800421204601F0EBF938B984F831A00A
:1074500002E0042084F83100C4F82094A07878B1C8
:107460003A4604F15400D4F8201472DF00287FF467
:1074700014AF94F8301094F8540073DF0028F6D15C
:10748000616B11B194F831008847002005E784F85A
:107490003150F5E710B5044600F006F808B1204673
:1074A00010BD142010BD0000142801D30020704727
:1074B0000146014801F0BDBC9CA600207CB50546F4
:1074C00008880C460930904201D90C207CBD6846E2
:1074D0006DDF0028FAD121880820685420881B21FC
:1074E000401C80B2208029542088401C80B220801B
:1074F0002844DDF801100160BDF805108180208866
:10750000801D80B220809DF80010490800D0012124
:1075100029542088401C208000207CBDF8B52B4DCC
:1075200001880446AE8821293BD015DC2848294A29
:107530001029A0EB02004FEAD0004FF0030202EB4B
:10754000004013D0112925D0132929D100231A4630
:10755000852130467FDF17E03B2932D052292AD0DF
:1075600056291DD18088132176DF0DE01AA102F083
:10757000E5F9072000F002FB08B1FFF7BDFBA18889
:10758000A980184801F094FD002809D0BDE8F84012
:10759000FFF7B2BB14A102F0D1F94FF6FF70A8803B
:1075A000F8BD00200090A08869468FDF0028F7D042
:1075B000FFF7A2FBF8BD00231A4619463046B1DF9B
:1075C000E2E78088132176DFDEE70000D82A00207A
:1075D00020BE0200B8BD0200436F6E6E6563746525
:1075E0006400000084A10020446973636F6E6E65BF
:1075F000637465640000000010B51A4C018860686F
:1076000010290ED011292BD1401E606028D1FFF720
:10761000B2FA002824D02168002921D0BDE810400A
:107620000847D0B900210122084600F085FA08B1C8
:1076300007280FD107220221012000F07DFA08B1AE
:10764000072807D104220221002000F075FA20B19A
:10765000072802D0216801B188476068401C60603B
:1076600010BD0000342B00202DE9F04701883B4E6F
:1076700040F2F3194FF6FF7510291BD011293ED0A7
:10768000122954D0502946D1C188F289841D9142D3
:1076900041D1618902293ED18688304601F00CF93A
:1076A000050038D004F10C0000F08DF9A8B329468C
:1076B00030464EE0C17B8788044601292BD1A8467D
:1076C000284601F0F9F8050017D02F800020287215
:1076D000234843464A460168C5F80A104068C5F881
:1076E0000E0004F1100105F10A0001F05CF9687266
:1076F000F08900280FD129462AE0042013E0808871
:1077000001F0DAF8040006D06068FFF771FB08B1F9
:1077100003F0E8FA2580BDE8F087FFE76868FFF727
:1077200067FB0028F7D0BDE8F04703F0DBBA878895
:107730000646384601F0C0F80400ECD02B464A4615
:1077400006F1080104F10A0001F02DF960722146EA
:107750003846BDE8F04700F0DDBD00007CA6002003
:107760003C2B00202DE9F04F0446868801884248D2
:1077700097B0834610290CD0112950D01030192908
:107780006AD01A2974D1217A0C09042C4DD3012214
:107790004CE0394D083DA868C0430B9069680BA8C0
:1077A00001F068FB0B990CA800F050FD2C220CA9ED
:1077B0006846FEF75BFE0027E946A84610E000BFDA
:1077C00009EB47005FF00005B0F804A008EB850066
:1077D0005146001D01F022FB6D1C1E2DF6D37F1CAF
:1077E0000098B842ECD8142E05D317B00420BDE899
:1077F000F04FFFF781BA3146584601F025FB31467C
:1078000008F1040001F020FBE07B022830D117B022
:107810003146BDE8F04F1848001D01F015BB17B008
:107820003146BDE8F04F01F0F9BA0022314600F0D0
:10783000F2FF032C01D3012200E000220E48314662
:107840000C3000F0E8FF022C01D3012200E00022FE
:1078500009483146083006E0217A002908D1617ACA
:10786000C1F3C002314617B0BDE8F04F00F0D3BFFE
:1078700017B0BDE8F08F0000A0A6002070B5334D12
:1078800004008EB02DCD08AE86E82D005BD0E9B3A4
:107890000868A061214608A862DF002851D120783D
:1078A00001258DF83200ADF83050A21C0CA92846F5
:1078B000A8DF002845D120216846FEF7F0FD022010
:1078C000ADF8000020788DF802008DF80C509DF87E
:1078D0000D00F426ADF8046040F00C008DF8115056
:1078E000ADF806508DF80D008DF81250608804F147
:1078F0000C02694600F0B4FB002822D12021684622
:10790000FEF7CDFD0320ADF8000000E01BE020787D
:107910008DF802008DF80C509DF80D008DF8115077
:10792000ADF8046040F010008DF81250ADF806502C
:107930008DF80D008DF813506088221D694600F007
:107940008FFB0EB070BD0E20FBE700003CB30200C1
:1079500070B588B00446002927D0002C25D00846F1
:107960002188102923D0502927D057291DD1054619
:10797000A188406906AAFFF7A9FA002815D1069E3A
:107980003078002811D0A86900280ED01821684648
:10799000FEF785FD01208DF800000195A088ADF867
:1079A00008000396A9696846884708B070BD08B00A
:1079B0002146BDE8704002F04EBE08B02146BDE849
:1079C000704002F027BF007800F00100704700000F
:1079D0000149085C70470000F4B2020007490B5CE3
:1079E0004FF0A041D1F804250120984020EA02037D
:1079F000C1F808351040C1F80C057047F0B202001C
:107A00000249085C012101F098BD0000F0B20200BB
:107A10000249085C002101F090BD0000F0B20200B4
:107A20000649095C4FF0A040D0F80405C84010F0AA
:107A3000010000D0012080F001007047F0B2020088
:107A400010B500242046FFF7DBFF641C042CF9D39B
:107A500010BD10B500242046FFF7DAFF641C042C8B
:107A6000F9D310BD10B50246064B4FF0FF30002190
:107A70005C5C944201D1084610BD491C0429F7D32F
:107A800010BD0000F4B2020010B5002000F066F94D
:107A900008B1062806D1012000F060F908B10628D7
:107AA00000D1002010BD00002DE9F0470D468146B1
:107AB000FFF7D8FF0446042836D2DFF874801B484D
:107AC0001C4EA8F10C0725B3012D0ED0022D2BD191
:107AD00004EB440030444578002D25D0B9680029D6
:107AE00022D02846BDE8F047084704EB4401755C06
:107AF0000E44717849B10E4A4FF48041093A8068CA
:107B0000FFF75EF908B987F80390B17808F8041018
:107B1000E2E78068FFF76CF904EB4401314418F8A0
:107B200004008D78A842D7D0BDE8F087F8B20200F3
:107B3000302B002018A6002070B50023042810D296
:107B40000D4D00EB4004012A02D101290CD0002286
:107B5000094E00EB4000304461B1012906D00229F2
:107B600006D00723184670BD0E30C2B22A55F9E779
:107B70004270F7E78270F5E718A60020044A014634
:107B800000201279D20702D0084600F003B87047EF
:107B9000242B00202DE9F05F6E4C0546002660780E
:107BA000B34618B184F801B000F020FF6A4F4FF4DB
:107BB0007A694FF4C87A4FF00108182D69D2DFE8CE
:107BC00005F00C1313384754696E727B727BC584C1
:107BD00084848484B3B6B9BCC5C500F007FF386897
:107BE000FFF706F906465CE00020FFF719FF0028C2
:107BF0004FF0000008D0FFF703FF022D02D14FF431
:107C0000E16008E0484606E0FFF702FF022D01D1DF
:107C1000C82000E05046410CC0034FF47A7280182F
:107C200041F10001257052000023FEF7DBFB014605
:107C30002AE00020FFF7F4FE00284FF0000004D0F7
:107C4000FFF7DEFE4FF44870E5E7FFF7E1FEDFE700
:107C50000020FFF7E5FE00284FF0000002D0FFF7FC
:107C6000CFFECFE7FFF7D4FED4E70020FFF7D8FE22
:107C700000284FF0000002D0FFF7C2FE01E0FFF73E
:107C8000C7FE257040F6CD4100223868FFF798F80E
:107C9000064646E00020FFF7A1FE257008E0002020
:107CA00051E025703DE084F801800120FFF796FE49
:107CB000002240F26661E8E784F801800120FFF7C6
:107CC0008DFE00224FF40051DFE77868FFF790F84F
:107CD0000646D5F1110000D02EB10220FFF790FE2C
:107CE00084F802B01DE0012816D980B2C8214843AB
:107CF000C117C90341EA5041C0034FF47A7280189A
:107D000041F1000152000023FEF76CFB0146002206
:107D10007868FFF755F806460220FFF779FE84F8E9
:107D200002803046BDE8F09F00F060FEB9E700F049
:107D30005DFEB4E700F05AFE04E000F057FE0020BC
:107D4000FFF766FE0120FFF763FEAAE7FFF781FE5B
:107D5000A7E70000242B0020F8B20200012103F065
:107D6000A8BA00002DE9F84F0546861C00208DF8C2
:107D7000000091460F464FF0010A6846FFF768F889
:107D80001B4C04F21C4860683860D4E90101194FAB
:107D9000401A3968081A0EE00121404601F064F8E3
:107DA00000F048FE0146404601F05EF8D4E90101CA
:107DB000401A3968081A401C8642EDD8B9F1000F04
:107DC00003D0052065F3891002E0062065F39F507B
:107DD00061683A68114004EB8101C8606068304412
:107DE00060609DF80000FFF757F85046BDE8F88F37
:107DF00054AA0020D02B002070B50D4604460A2955
:107E000002D10D21FFF7F8FFA0682268411CA16094
:107E10001554D4E90101814204D32046BDE87040E5
:107E200001F025BA70BD00000448816840688142B5
:107E300001D10120704700207047000054AA0020A3
:107E400010B51A280ED101290CD10748002240F2A2
:107E500066610068FEF7B4FF002803D0BDE810405B
:107E6000FEF74ABF10BD0000ECB20200034630B579
:107E7000074800210478426806E000BF02EBC10019
:107E800005789D4203D0491CA142F7DB002030BD9C
:107E9000602B002070B50020FEF7DAFE2149224A4F
:107EA0000026891AC9080322204C02EB0145D8B1EB
:107EB0002069401C2061142809D328461CA1266192
:107EC00001F03CFDBDE87040132001F028BB1D48C7
:107ED000002240F266610068FEF772FF00281CD0A5
:107EE000BDE87040FEF708BF2661606916A1401C1E
:107EF0006061284601F022FD606902280DD12078DA
:107F000060B1012809D1284614A100BF01F016FD77
:107F10002078C0F101002070666170BD284617A16D
:107F2000F4E7000020BE0200B8BD0200D82A0020FD
:107F30004C6F6E6720427574746F6E20707265733B
:107F400073000000ECB2020053686F727420627517
:107F500074746F6E207072657373000053746F7069
:107F600070696E6720736176652064617461207446
:107F70006F205344636172640D0A00005374617290
:107F800074696E6720736176652064617461207422
:107F90006F205344636172640D0A00000F4810B5EE
:107FA0001A2101700E4941600121817041706422E3
:107FB000FEF70EFE08B1FEF79FFEFEF7F7FD08B1D3
:107FC000FEF79AFE074A00210748FEF7BFFE002889
:107FD00003D0BDE81040FEF78FBE10BDF42A00208C
:107FE000417E0200957E0200ECB2020005494FF08E
:107FF000FF32082841F8202002D3084480F84820A6
:108000007047000028A70020F0B54FF0FF3512B1EF
:108010000023082601E008230C260C4C05E000BFD5
:1080200054F823707F1C04D05B1CB342F8D328465D
:10803000F0BD26185DB286F8305044F82310002AAF
:10804000F5D1E11881F84800F1E7000028A70020E9
:108050000249084490F930007047000028A700202A
:108060002DE9F0438146887891B090460C4600B9DE
:1080700001208DF83E002088ADF83C0000250095D9
:10808000607C694602F0A2FE6E46A07C711C02F084
:108090009DFEE07B00289DF8020002D040F0080021
:1080A00001E020F008008DF80200217C11B140F0C1
:1080B000100001E020F010008DF80200217B11B1CA
:1080C00040F0010001E020F001008DF80200217D68
:1080D00009B1022100E0012161F342008DF80200A4
:1080E0001C2102A8FEF7DBF9607BC10601D48006E3
:1080F00017D50E950EAFE07C791C02F067FE9DF857
:108100003800079720F00F00401C20F0F0001030DE
:108110008DF838009DF83A0020F00600801C8DF89C
:108120003A00607B8DF80800A07B8DF809001421CF
:1081300009A8FEF7B4F90FA8CDE90906A088ADF8A3
:108140003000A06820B1E088ADF82C00A0680D9048
:10815000A06998B301950088ADF81000A06901AD41
:1081600001A94088ADF81200A06940680695039007
:10817000A069007B02F02AFEA069691C407B02F026
:1081800025FEA069807A00289DF8060002D040F004
:10819000080001E020F008008DF80600A169C97A06
:1081A00011B140F0100001E020F010008DF8060041
:1081B000A169097A19B140F0010002E00DE020F058
:1081C00001008DF80600A169897B09B1022100E058
:1081D000012161F342008DF80600E06900B10590CD
:1081E000434609AA02A94846AADF11B0BDE8F083B8
:1081F00070B5084C050009D010342168002907D05B
:1082000008682060496828468847F6E70834F4E79C
:1082100070BD000014A70020054A012120B10128EB
:1082200005D19170FFF7E4BF51700020FAE7704765
:1082300014A7002010B5D0E90234D1E90220D11AE8
:10824000A04101D3012010BD002010BD73B58CB03A
:108250000646002000900D9880B100246D4621460E
:108260000DA800F0E6FD30B1009805EB40008480D9
:108270000098401C0090641C142CF0D32C226946FA
:108280003046FEF7F3F80EB070BD2DE9F0411788C7
:108290000646B81D14460D46984202D90C20BDE88A
:1082A000F0813188072206290AD34FF4486C4FF633
:1082B000FF73614501D9994202D17088062801D225
:1082C0001046ECE7604501D99842F9D1994203D0B4
:1082D000984201D08142F3D80520E8552088122128
:1082E000401C80B2208029542088401C80B220800D
:1082F0004119308802F0E8FE2188084480B22080CD
:108300004119708802F0E0FE218808442080002096
:10831000C5E7000038B54A7A0F4B62B100220A72F5
:108320005969002906D001228DF80020ADF802001D
:108330006846884738BD0A7A62B19B684C68024635
:1083400019462046FEF73CFD0028F3D0BDE8384032
:1083500002F0C8BC5B68F1E77CA6002070B588B06D
:108360000646002005900690ADF81410ADF81610E2
:108370000190029001AA05A9304690DF050021D0A6
:1083800001F0B4FE0346114811493246401AC108B3
:10839000012000EB014004460E4901F0DAFABDF875
:1083A000042012B9BDF8060028B1BDF806302046F9
:1083B00009A101F0CEFABDF808201AB120461649ED
:1083C00001F0C0FA08B0284670BD0000B8BD020038
:1083D000B8BD020010B60200546865207265717560
:1083E00065737465642054582F5258207061636B14
:1083F0006574206C656E67746820697320746F6F94
:10840000206C6F6E672062792025752F2575206F8F
:1084100063746574732E00005CB6020070B50024AE
:108420000F4D10E0686800EBC406307801F082FF61
:108430007178012901D0012100E00021414030780C
:1084400000F05CF9641C28788442EBDBD5E9040178
:10845000084303D0BDE8704002F01ABE70BD0000B2
:10846000602B002010B50021024800F00EFD80F3C3
:10847000100010BD70AE00204FF480328A400168B9
:10848000C1F848230068C0F8082370474FF4A07271
:1084900002EB810189B200F0A1B92DE9F041054656
:1084A0000E464FF4A07000EB860081B228684FF4AE
:1084B0008034B440984622F07F47C0F808432868CB
:1084C000C0F84843286801F0BEFB286800EB86002E
:1084D000C0F840752868C0F84443B8F1000F02D0D6
:1084E0002868C0F80443BDE8F0810068D0F80405AE
:1084F0007047000070B54379234C44F8232042793B
:10850000231D03EBC202224C1579204A121BD4080A
:108510002DB10825022000EB04401EA130E00568C3
:108520000A88C5F8082590F904208978002A4FEABE
:10853000411104DB02F1E02282F8001405E002F0B0
:108540000F0202F1E02282F8141D90F904100122BA
:10855000002909DB01F01F0502FA05F54909890028
:1085600001F1E021C1F800514179002503EBC1017F
:108570000A71417943F83100032000EB04400EA159
:1085800001F0DCF9284670BDB82B002008BE0200BF
:10859000B8BD020052544320696E7374616E636506
:1085A00020616C726561647920696E697469616CBF
:1085B000697A65642E0000005254433A20696E695E
:1085C0007469616C697A65642E00000090F904009A
:1085D000002809DB00F01F020121914040098000C2
:1085E00000F1E020C0F8001270470A46022100F0B6
:1085F0007BB84FF4827100F0F1B80068012101608E
:10860000704700680121416070472DE9F05F07461F
:108610000C464FF4A07000EB84001FFA80FA386813
:108620004FF48036A6409B4622F07F45C0F8486351
:108630003868C0F808633868D0F8048500EB840215
:10864000D2F84095C2F840855146386801F0FBFAEF
:10865000A9EB080020F07F40012806D1102001F08E
:10866000ABFD5146386801F0EEFA3868D0F8048561
:10867000C0F84463A5EB080121F07F413868012967
:1086800000EB840010D0C0F840553868D0F80415CD
:108690006FF07F4C6A1A521E22F07F42ACEB0B0344
:1086A000934217D362B118E06D1CC0F840551020FA
:1086B00001F082FD3868D0F8040540450AD10CE08D
:1086C00000EB84006D1CC0F840553868D0F80405F4
:1086D000884202D00D20BDE8F09F01223146384685
:1086E00000F002F80020F6E70368C3F84413002AFC
:1086F00002D00068C0F80413704700002DE9F84F5D
:108700000E463449804601EB5001C007097801D07C
:108710000F0901E001F00F074FF000094246012068
:108720004946FDF790FEDFF8B0A004460D46052F40
:108730004ED2DFE807F003161B282C00002E47D08E
:108740000121404602F098FB8DF800906846FEF744
:108750007FFB5046D0E904120C431543CAE9044597
:1087600032E00EB1022114E0002112E04EB10321EB
:10877000404602F081FB4046BDE8F84F012102F07F
:1087800021BD012105E0002E22D1042101E02EB1FE
:1087900003214046BDE8F84F02F06EBB0021404681
:1087A00002F06AFB0021404602F00CFD8DF80090BB
:1087B0006846FEF74DFB5046E243D0E904341A40C8
:1087C00024EA0501CAE904219DF80000FEF764FBD4
:1087D000BDE8F88F18A80020602B002010B50068B5
:1087E00042581AB101F02FFA012010BD002010BD2F
:1087F000826883881A4003689A5C0A708168491C01
:1088000081607047C26883881A4003689954C168C0
:10881000491CC16070470AB100F016BB00F0FEBAF7
:1088200070B50D460446B0F81414D0F810040122B7
:10883000FEF731FC00B1057004F13C0204F58261E1
:1088400004F1540072DF70BD10B50B48FFF74DFE08
:10885000094A083AD2E90434C018D2E9063244F190
:108860000001C31A71EB020204D24FF0807280182B
:1088700041F1000110BD0000802B002010B5C0B2F6
:10888000FFF7F4FA0446007801F054FD01466078E1
:10889000012801D0012000E0002090EA010F08D05B
:1088A0000449D1E90401084303D1BDE8104002F0B6
:1088B000EFBB10BD602B00200146034802888A42AE
:1088C00000D000207047000068A600202DE9FC5F62
:1088D0000E008346DDE90C47C6F10000984692463B
:1088E000814600D40846012503E000BF90FBFAF062
:1088F0006D1C5045FADAA84500D9454624B1002E32
:1089000001DB780700D5641EB80702D5B8F1000F67
:108910000AD0F80708D13CB1A54205D2202158461B
:10892000641EFFF769FAF6E7002E02DA4E462D21A3
:1089300002E0780703D52B215846FFF75DFA07F0D0
:10894000030002280BD1B8F1000F08D13CB1A542B9
:1089500005D230215846641EFFF74EFAF6E7CDE9FE
:108960000047434652463146584602F0B3FBBDE845
:10897000FC9F024600201268530713D502F0030043
:10898000012802D002280CD105E0C2F383100B6845
:10899000801C184404E00223086803EB9252104440
:1089A000086001207047F0B58488A518944200D86B
:1089B0002246A41AC288D6189A4200D81346D21A60
:1089C0004B880788BB420CD34088834209D88888EB
:1089D000A04206D3A84204D8C888904201D3B0422E
:1089E00001D90020F0BD0120F0BD00000A4810B5FB
:1089F000807860B1002401E0022C06D02046FEF70A
:108A0000FFFF641C042CF7D310BD0324F6E7BDE878
:108A10001040FFF715B80000242B0020F72101803B
:108A200017214180002101714171FB2181711B21BE
:108A3000C17170472DE9FF410026244800F011FA6A
:108A40002248001F074600F00CFA214C2149A0687B
:108A500000900D6800E000986946284004EB800013
:108A60000C30FFF786FF0028F5D101AA009901EA32
:108A7000050304EB8303491CDB6842F82030401CEB
:108A800000910228F2D3019800F0030001280BD0D6
:108A9000022810D10198032101EB90500099BDF8F4
:108AA0000A6001EB900005E00198BDF80A60C0F390
:108AB000831008440090384600F0D0F908B10098BF
:108AC000A06004B03046BDE8F08100006CAE00202C
:108AD00054AA0020D02B0020ACB0042000F0D2FC1F
:108AE000132000F0CFFC4FF0A0410125E804C1F8AD
:108AF00008054111002000F08DFF08B1FEF7FCF8D9
:108B000000F0F2FDFEF72EF908B1FEF7F5F802F0DD
:108B100041FA01F009FA08B1FEF7EEF800246946BF
:108B20000120009401F0A0F808B1FEF7E5F86846CE
:108B300001F032F908B1FEF7DFF82548019001A9EC
:108B4000244800F0C0FA08B1FEF7D6F82248009099
:108B500069462248FEF792FE08B1FEF7CDF8AC2137
:108B60006846FDF79CFC02208DF800008DF802405D
:108B700005208DF803001948ADF84C5018381490B2
:108B80004020229044F2506023908DF87C5014488D
:108B90002990104869460C30FEF7B3FA08B1FEF789
:108BA000ABF80C4801210C30FEF7A8FAFFF7F6F9F4
:108BB00002F008F8094D4FF47A76243DA868B042D7
:108BC000FCD1042000F0ABFCAC606C80F6E7000048
:108BD000279C020084A1002071A50200FC2A00202D
:108BE00021A6020070B5144682880E4605462088EC
:108BF000111D0144921C994201D8FE2A01D90C2072
:108C000070BD521C32542088FF21401C80B220804D
:108C100031542088401C80B220808119288802F0BD
:108C200053FA2188084480B22080AA8842B1A968FA
:108C300041B13044FDF71AFC2088A98808442080FF
:108C4000002070BD072070BD2DE9F047C5881E1DAE
:108C5000B6FBF5F78946B6FBF5F1044605FB176C44
:108C6000407916686843DDF820A0F718001F874296
:108C700000D9C61A166001E02468491E0029FBD1FC
:108C8000A5EB0C078846B74216D818E004EB0C0099
:108C9000001D09EB0803BAF1000F3A4602D0014665
:108CA000184600E01946FDF7E1FB2468F61B4FF07B
:108CB000000CB844B54201D9374600E02F46002EDB
:108CC000E4D1BDE8F087000030B5024651B100F0B4
:108CD000B5FE0021074C08E034F821301568AB429E
:108CE00002D11160002030BD491C8142F4D305201F
:108CF00030BD000000000000F8B50F4601781446B2
:108D00000546012901D1687830B12088821C9A4239
:108D100032D8012902D006E00720F8BD6978014465
:108D2000891C994228D8181A801E86B2ADF80060B6
:108D30002188B81C084469467DDF0028EDD12978D8
:108D4000022904D06878BDF80020904205D3BDF810
:108D50000000B04201D809200AE00820012905D10D
:108D60006978B14202D8ADF8001001E0ADF80060BA
:108D7000BDF80010FE2901D90C20F8BD2288491C3D
:108D8000B9542188491C89B2218078542088401C1C
:108D90002080BDF80010084420800020F8BD10B5E8
:108DA00031B1B2FBF3F403FB14241CB1092010BD54
:108DB0000E2010BD01600021416081608281C3816D
:108DC000084610BD70B50C460546FDF723FA00288D
:108DD00002D021882868084470BD10B50A884988E7
:108DE0008A4203D1FDF758FA012010BD002010BDC2
:108DF00070B50C460546FDF732FA002802D06188AE
:108E00002868084470BD10B50A8849888A4203D191
:108E1000FDF71CFA012010BD002010BD01F01F035A
:108E200001229A40D243490900EB8100114600F02B
:108E300021B84A0950F8220001F01F020121914097
:108E4000084000D00120704701F01F0301229A4022
:108E5000490900EB8100114600F01CB8002100F028
:108E60000FB8012100F016B808B56A46FDF769FA97
:108E7000009808BD08B56A46FDF749FA009808BD94
:108E800008B56A46FDF743FA08BD08B56A46FDF71E
:108E900025FA08BD08B56A46FDF72CFA009808BD0A
:108EA00008B56A46FDF75AFA009808BD38B5044679
:108EB00000258DF800506846FDF7CAFF21686268FA
:108EC000086890420ED9401E08600178238AE26843
:108ED00001FB0325227A2168101AC0B20A79824266
:108EE00000D208719DF80000FDF7D6FF284638BD76
:108EF00038B5054600208DF800000C466846FDF7A1
:108F0000A7FFE868298A201AB0FBF1F12A681068E7
:108F1000431C136001709DF80000FDF7BDFF38BDD4
:108F200010B530B1017A42680368891AC9B21A6073
:108F300006E00E2010BD03681A68541C1C601170F6
:108F4000491EC9B2F7D2006800210171084610BD60
:108F5000C20800F007030120895C98400840704770
:108F6000F0B5858893B00C46002D39D101880026D4
:108F70003F4F24293BD006DC102909D011290CD001
:108F8000232958D14FE03A290BD0552953D129E054
:108F90000146204601F094FB4DE0A01DFFF73EFD89
:108FA00049E02246408934F8061F814200D808462D
:108FB0006080172800D217206080106970B1607936
:108FC00060B1D7E90001CDE90301ADF80E5060882A
:108FD000ADF81000136903A9104698476671267111
:108FE00013B0F0BD0146204601F0BEFB23E0011D99
:108FF0002C2206A8FDF73AFABDF81800BDF81C208F
:1090000004EBC0014A732269AAB1D7E90423CDE970
:109010000423ADF81200487B8DF814002269204625
:1090200004A9904707E0017A207B884200D20146DC
:109030002846FFF793F9A07A0028D1D0E188284686
:10904000A5DF012580B11128CAD001F04FF80246F2
:109050000848094913B0401AC00805EB0040BDE8B4
:10906000F04006A100F06EBCA672E572B8E7000001
:1090700024B30200B8BD0200B8BD020073645F6291
:109080006C655F67617474635F65786368616E6760
:10909000655F6D74755F72657175657374282920DD
:1090A00072657475726E65642025732E0000000071
:1090B00020B10278DE2A03D0082070470E207047C6
:1090C00041800020704760B159B10278DE2A0AD091
:1090D00009684160DE2101704FF6FF714180002078
:1090E00070470E207047082070477FB5054600295D
:1090F0004DD0002D4BD008780C46DE2847D1A888EB
:109100006188884202D1204602F04AF82888012866
:1091100025D002283BD011283AD0512837D135F834
:10912000040F6188884232D1A978A81C02292ED167
:10913000017A042903D0062901D0052927D100216D
:10914000009102228DF8002001914FF4C07202912B
:109150000391ADF80420007A05280FD010E0297A99
:109160002046012913D1A988428891420FD10121BB
:10917000017204B0BDE8704002F012B8ADF80410FE
:1091800028886946B0DF002801D0616888477FBD24
:10919000A88861888842FAD14FF6FF7060807FBD51
:1091A00000F180400068002800D00120704708B519
:1091B00000F18040002101600068009008BD0000BF
:1091C00070B50D4C0125207808B185260EE00020F1
:1091D000A06060602061E060084800F0C5FF0646BE
:1091E00000F0EEFE08B900F0A9FF257000F09EFF28
:1091F00000B1A570304670BD14A70020198202008E
:1092000038B500258DF800506846FDF721FE084C62
:10921000E068401EE060E06828B900F087FF10B900
:1092200000F0B2FFA5709DF80000FDF735FE38BDD7
:1092300014A7002030B40378054CE35C1BB130BCAC
:10924000001D01F031B930BC0C3001F0C9B800008C
:10925000442B00200FB408B50399002904D004AAB8
:1092600000926A4600F00FF801B05DF814FB10B5EB
:1092700082680446002A05D0D4E90403216898478F
:109280000020A06010BD2DE9FC4791460C008046EF
:1092900076D014F8011B39B125290ED04046FEF7CF
:1092A000ABFD20780028F4D198F80C00002867D096
:1092B0004046BDE8FC47FFF7DABF002001222178D5
:1092C0002B291BD02D2902D0302908D102E040F0F3
:1092D000010001E040F00200641C002AEFD10025EB
:1092E0002A290ED02178A1F130020A2A11D205EBE9
:1092F000850201EB4205641C303DF1E740F00400BB
:10930000EAE7D9F800100B1DC9F800300968641CA1
:109310000D44217800232E290BD114F8011FA1F14F
:1093200030020A2A05D203EB830201EB4203303BF1
:10933000F3E76C290DD068290BD0692921D00BDC0B
:10934000252918D0582931D063290ED0642915D188
:1093500017E014F8011FECE7702969D0732932D0A7
:1093600075291BD0782909D120E0D9F80000011D0A
:10937000C9F8001001784046FEF73EFD641C90E7F6
:109380006CE0D9F800100A1DC9F800200968CDE981
:1093900000500A224046FFF799FAEFE7D9F800108B
:1093A0000A1DC9F8002009680A2206E0D9F8001051
:1093B0000A1DC9F8002009681022CDE90050404676
:1093C00001F088FEDAE7D9F8001000270A1DC9F875
:1093D00000200E68C00705D112E04046761C7F1CB5
:1093E000FEF70AFD31780029F7D104E0202140463C
:1093F0006D1EFEF701FDBD42C0D9002DF6D1BDE7BF
:109400004EB13046FDF756F8074604E020214046AD
:109410006D1EFEF7F1FCBD4206D9002DF6D103E02A
:109420004046761CFEF7E8FC31780029F8D1A5E724
:10943000D9F80000011DC9F8001005683021404628
:10944000FEF7DAFC78214046FEF7D6FC0820002122
:10945000CDE90001034610222946B0E7BDE8FC87AC
:1094600070B541EA4201DDE904564FF0A04441EAFB
:10947000830141EA052104EB800041EA0641C0F87E
:10948000001770BD4FF0A04202EB80000321C0F82E
:10949000001770474FF0A04202EB8000D0F8002781
:1094A00022F44032C0F80027D0F8002742EA0141F8
:1094B000C0F800177047000038B5094B44181B6806
:1094C00000936B4608E000BF53F82010D1F82055F8
:1094D00020C2C1F82055401C8442F5D838BD000098
:1094E0004CB302004FF0A04201218140C2F80C159C
:1094F000704742094FF0000100D1491E00F01F00E3
:10950000012282400A4201D00120704700207047AA
:109510004FF0A04201218140C2F8081570474FF07A
:10952000A042D2F804350121814021EA0300C2F8AB
:1095300008051940C2F80C15704701224FF0A043EE
:10954000824011B1C3F808257047C3F80C25704755
:10955000034908B50844002101600068009008BD77
:109560000060004002494058012800D000207047A8
:109570000060004030B5154A01460020D2F8104482
:1095800023460AE0DB681D79854205D1401C0A2884
:10959000F6DB4FF0FF3030BD1B68002BF2D1431CCF
:1095A000F9D0CB681871D2F8103443B1DB68CC68BD
:1095B0001B682360D2F81024D268116030BDC2F855
:1095C0001014C96800220A6030BD000054AA0020AF
:1095D0007047FDF769B8704708B5034A0092402309
:1095E000024A00F005F808BDF5AC0200BCA8002056
:1095F000F0B595B01C4615460F4608461A9E00F079
:10960000EDFA182109A8FCF74AFF0E96CDE9095496
:109610000023082203A9384600F0F5FA05980690C1
:10962000BDF81000ADF81C00BDF81200ADF81E002A
:1096300000208DF821000398082600F0030001287F
:1096400002D0022818D032E003983346850AC0F3CE
:10965000C2008DF8200003980FA9C0F38314A20064
:10966000384600F0D0FA09A8009006AB22460FA9B0
:10967000284600F00FFA1AE00398840DC0F3C200E8
:109680008DF82000082C01D2254600E0082533463D
:109690002A460FA9384600F0B6FA2E44641B09ABDF
:1096A00006AA29460FA800F05DF9002CEAD1384639
:1096B00000F09AFA15B0F0BD0A4A012902EBC00089
:1096C00007D0022907D0032907D0042907D000209A
:1096D0007047022070470420704700797047407936
:1096E00070470000B8BD020010B5FFF772FF0421FB
:1096F0000348FFF73FFF02490120C968487110BDC8
:10970000A8BD02002DE9F04F8DB0FEF78DFB18B11A
:1097100000200DB0BDE8F08F7E4C4FF0000BC4F878
:1097200018B4BFF34F8F7C49A06802900D68D846EB
:10973000284004EB80000BE0D4F8180470B961688D
:109740000298814201D8A160E2E7284004EB800042
:109750000C3002A9FFF70DF90028EDD1002005AA71
:10976000029901EA050304EB8303491CDB6842F814
:109770002030401C02910228F2D3059800F003002B
:10978000022802D001284DD0AAE005985022810D70
:109790008946B2EB905F00D850210E4666F39F5089
:1097A000059008315D4800F0D0F9070078D000F04E
:1097B00015FA4346082205A9384600F02CFA02990A
:1097C00008F1080A2940681A8000001D864222D943
:1097D000504D0C3530B1C2B204EB8101301A9046C5
:1097E0000C3104E02946F2B2002590462846C6B264
:1097F0005346384600F00FFA0AEB080325B132460B
:109800002946384600F007FA029909F1030001EBF6
:10981000900002903BE004EB81015346324638460B
:109820000C31EFE70598C0F38310062800D306201B
:10983000059960F38911C1F38310801C05918100A3
:10984000364800F082F907004AD000F0C7F94346D5
:10985000082205A9384600F0DEF908F108080026BC
:109860000FE00298434600EA0501401C04EB810129
:109870000290042238460C3100F0CDF908F10408BA
:10988000761C0598C0F38310B042EAD847B1D4F8EB
:109890001054D4F8180478B1384600F0A5F934E033
:1098A0001EE0E8684079012804D12A682846394634
:1098B00012689047E8680568002DF2D1384600F03C
:1098C00093F98DF800B06846FDF7C2FAD4F8180491
:1098D00008B90298A0609DF80000FDF7DDFA14E0D9
:1098E000D4F8104405E02168204689688847E0687C
:1098F0000468002CF7D10A480A49401AC00802211E
:1099000001EB004008A100F019F8FEF78DFA80F095
:109910000100FEE654AA0020D02B002040BE020029
:1099200020BE0200B8BD02004261636B656E6473C5
:1099300020666C75736865640000000000231A4699
:1099400001F0B2BA08B5012300926A4601F0ACFA00
:1099500008BD1CB5CDE9002302236A4601F0A4FA34
:109960001CBD00002DE9F0470E4680461C4692467D
:10997000082940D894F80C9000202073194610460E
:1099800001F03AF80025B54206D218F805201BA1CF
:109990002046FFF75FFC03E01AA12046FFF75AFCC0
:1099A0006D1C082DEFD318A12046FFF753FC0025AE
:1099B000B54212D218F805707E2F08D8FCF752FD78
:1099C0000068C05D10F03E0F01D03A4600E02E2244
:1099D0000EA12046FFF73EFC03E00DA12046FFF755
:1099E00039FC6D1C082DE3D301222146504600F0BE
:1099F000E5FF84F80C90BDE8F087000020253032A8
:109A000078000000202020007C000000256300007A
:109A100020000000064910B501200870054800F03C
:109A2000E1F8002803D1044800F0FFF8002010BD41
:109A300054AA002040BE0200D8B4020002480349E4
:109A4000401AC0087047000040BE0200B8BD0200C6
:109A500013B56846FFF738F908B100201CBD02486D
:109A6000009950F831001CBDB8BD020070B508481F
:109A70000125D0F81044057007E0E06845712168C1
:109A8000204649688847E0680468002CF5D170BD1D
:109A900054AA00202DE9FF4781460C9D00200C466A
:109AA0002F7B2873984616462946184600F0A4FFD7
:109AB000072E42D2DFE806F004090F161F2A3600EF
:109AC00049462846FFF7C6FB37E049462846226844
:109AD000FFF7C0FB31E0D4E9002349462846FFF7F1
:109AE000B9FB2AE0A0680090D4E900234946284643
:109AF000FFF7B0FB21E0D4E90201CDE90001D4E990
:109B0000002349462846FFF7A5FB16E004F10800AC
:109B100007C88DE80700D4E9002349462846FFF727
:109B200099FB0AE004F108000FC88DE80F00D4E9A2
:109B3000002349462846FFF78DFB00222946404670
:109B400000F03CFF2F73BDE8FF872DE9F041058A47
:109B500080462D1F4819C01CB0FBF5F0C6B2404628
:109B6000FFF7A4F9041E19D00020207101206071B4
:109B7000E58000272546761EC4F800800BE04046AD
:109B8000FFF794F960B16179491C6171286005465D
:109B90007F1CC0F80080B742F1D32046BDE8F081B9
:109BA000204600F002F80020F8E72DE9F041457961
:109BB00001466B1E002201E00968521C9A42FBD349
:109BC0000F680146002605E038460C68FFF790F95B
:109BD0002146761CAE42F7D3BDE8F0810121001D7D
:109BE000FFF742B9FFF79CB910B504460121001DEB
:109BF000FFF756F910F0FF0F04D12046BDE81040E2
:109C0000FFF7D3BF10BD1CB501920122009201AA3B
:109C1000FFF71AF81CBD1CB501920022009201AAA0
:109C2000FFF712F81CBDFDF767B88268002191604C
:109C300082681161826851618268D1608268516076
:109C400080680160704708B500224250405800907B
:109C500008BD000020B10349096801600020704779
:109C60000E2070475CB502002DE9FE4307460E4604
:109C70000846FFF7EFFF00287CD1002400940194F0
:109C800006208DF800704FF00108ADF80400029432
:109C90008DF8028069462020326869DF3649374AEC
:109CA000891AC908012202EB014530B100F01EFA01
:109CB000024628463249FFF745FE00948DF80180A0
:109CC0008DF80240019402948DF8034069464020CB
:109CD000326869DF30B100F009FA024628462949A6
:109CE000FFF730FE00948DF80070F720ADF8020009
:109CF0000194029469462320326869DF30B100F094
:109D0000F5F9024628462049FFF71CFE009401940D
:109D100002948DF8008069460120326869DF30B115
:109D200000F0E4F9024628461849FFF70BFE4FF40D
:109D3000B0600090019402946946A120326869DF06
:109D400030B100F0D3F9024628461149FFF7FAFD79
:109D50000094019402948DF800406946A020326876
:109D600069DF30B100F0C2F9024628460949FFF721
:109D7000E9FD0020BDE8FE8330BE0200B8BD020050
:109D8000FCBB020044BC020090BC02005CBB0200B1
:109D9000A8BB020008BB02002DE9F0410546076898
:109DA00060DF804619491A482A68081AC608BA426C
:109DB00019D9022000EB064416A12046FFF7BEFD8C
:109DC00020463A461FA12B68FFF7C3FD4FF0805095
:109DD000D0F80C012968800200F10050421A204698
:109DE00025A1FFF7AFFDB8F100004FF001040AD044
:109DF00000F07CF9024604EB06402AA1FFF7A2FD21
:109E00004046BDE8F0812F480470F9E730BE0200FB
:109E1000B8BD0200496E73756666696369656E74E4
:109E20002052414D20616C6C6F63617465642066E3
:109E30006F722074686520536F6674446576696339
:109E4000652E00004368616E676520746865205266
:109E5000414D207374617274206C6F636174696F1B
:109E60006E2066726F6D203078257820746F2030F8
:109E70007825782E000000004D6178696D756D20A1
:109E800052414D2073697A6520666F72206170704F
:109E90006C69636174696F6E20697320307825780E
:109EA0002E00000073645F626C655F656E61626CBA
:109EB0006528292072657475726E65642025732E7D
:109EC00000000000272C002030B51548ADF5017DBD
:109ED0000078002821D04FF4FA7500BFADF8005289
:109EE00080A9684661DF38B1052816D00DF5017DDF
:109EF000BDE83040FCF700BF6C460A497DA800F081
:109F000083F806E0D0E90021204690477DA800F0C4
:109F100092F87F980028E1D0F4E70DF5017D30BD7F
:109F2000272C002060B502007CB5194C207808B1C0
:109F300008207CBD0120A070002000F0A5FE1128A3
:109F400019D0002000F0B8FE1248002600680190E9
:109F50008DF800606846FCF77BFF0F4901A810DF11
:109F600005000AD0002020709DF80000FCF794FF47
:109F70002DB128467CBD00207CBD0120F3E7A670F2
:109F8000667000F047FF012000F096FEF3E7000046
:109F9000242C0020F4B40200756C02000EB50749B1
:109FA000684600F031F805E0D0E9001088476846BF
:109FB00000F041F802980028F6D10EBD10B502005D
:109FC0000148007870470000242C00201FB5684627
:109FD0004BDF30B1052814D004B0BDE81040FCF7C9
:109FE0008BBE084901A800F00FF806E0D0E9002177
:109FF0000098904701A800F01EF803980028E6D0CA
:10A00000F4E71FBD7CB50200016009684160AFF351
:10A01000008010B5D0E900215368994201D1002198
:10A0200004E0D1E90034A34202D01946816010BD9A
:10A0300008314160F0E7816800290BD0026892681E
:10A040000A44826041684B689A4203D108314160FA
:10A05000FFF7DFBF704770B50D460646446804E061
:10A06000B2682946904718B1246820680028F7D1C3
:10A0700020682860256070BD4068006870474168AE
:10A080000868002801D002680A6070470246002074
:10A09000526806E08B4203D10868106001207047C7
:10A0A0001A461368002BF5D170474058002800D09D
:10A0B000012070470C4A10B502F594730EE0991A0E
:10A0C000C91001EBD171491002EBC1010C68844247
:10A0D00001D90B4602E005D201F108029A42EED303
:10A0E000002010BD486810BD9CB3020000B5FFF70A
:10A0F000E1FF002800D1014800BD000088B3020044
:10A100004058002800D00120704708B50022425076
:10A110004058009008BD4058002800D001207047EA
:10A1200008B5002242504058009008BD024800681F
:10A13000002800D001207047000401400848006852
:10A14000012110F0010F06D14FF0E020C02280F86D
:10A1500000248430C1670349012008607047000073
:10A1600000E100E0180500400649024600200B7996
:10A170000BB1852070470A6001220A7100224A71E2
:10A1800070470000502B0020022010B54107C1F895
:10A1900008034FF48270FFF70AF8054901200860B0
:10A1A00004480168C1F300410029FAD110BD000044
:10A1B0000C00004018040040002802D00149800132
:10A1C0000847704771B302002DE9F0410E4605467D
:10A1D00000F07AFB0028284619D0FDF739FF08382F
:10A1E00000F0E4FB032802D001280ED007E04FF076
:10A1F000A040D0F81005E84010F0010F05D0032171
:10A200002846BDE8F041FFF745B90221F8E700F024
:10A2100067FB002822D02846FDF71AFF04464FF4BA
:10A22000807000EB84000E4F81B207EB8400D0F801
:10A23000102542F00102C0F810250846FFF788F902
:10A24000002E0BD02846FDF703FF064951F82000E9
:10A25000002803D00120A040C7F80403BDE8F08126
:10A260000060004028A700202DE9FC41DFF8B880FD
:10A27000044608EB0400002790F930001346C0178D
:10A280000E46401C01D008274AE0B0781946C0F3BA
:10A2900040022046FDF7B8FE0546401C3FD0B0788E
:10A2A000410717D4C0070AD04FF0A04000EB84004C
:10A2B000D0F8001721F00201C0F8001707E00021D4
:10A2C0007378204600910A460191FFF7C9F82046AD
:10A2D00000F0ECFAB078800718D51448317800EB1C
:10A2E0008500D0F81025124B1A40C0F810254FF405
:10A2F000F8524FF4403302EA042203EA01410A43D0
:10A30000D0F810150A43C0F8102509E008EB050045
:10A31000327810F8481F41EA8211017000E00427EA
:10A320003846BDE8FC81000028A7002000600040FE
:10A33000FFE0FCFF4FF0A041D1F81015C14011F033
:10A34000010000D00120704770B5194D95F85800F4
:10A3500008B1082070BD0024661E2046FFF7C9F82A
:10A3600010B1281980F83060641CE4B2202CF4D3BA
:10A3700000242046FDF73AFE641CE4B20C2CF8D30E
:10A3800000200D4968650B4CC02081F800040126AF
:10A390004020891FC1F800014FF4BE70FFF7D8F8C4
:10A3A000A004C4F8040385F85860002070BD0000C4
:10A3B00028A700200060004006E000E0034890F875
:10A3C0005800002800D001207047000028A7002076
:10A3D0000121B1EB507F01D101207047002070476F
:10A3E0002DE9F05F054600790B4600EB400101EBDB
:10A3F000C000244901EB8004284600F045F810B164
:10A400001120BDE8F09F62614FF00009C4F8209070
:10A41000A36084F828904FF48E784E464146286811
:10A42000FFF773FE28684FF0010AC0F808A0214624
:10A43000286800F039FE606808BBD5F800B067698D
:10A440000FE000BF94F8280008B10F2615E0414640
:10A450005846FFF755FE0028F4D02146584600F034
:10A4600023FE206AB842F2D3574641462868FFF7D8
:10A4700047FE0028F9D02868C760C4F81490304619
:10A48000BFE7000084A70020007900EB400101EB4A
:10A49000C000044901EB80004069002800D0012081
:10A4A0007047000084A700202DE9F04704460E46BF
:10A4B0000079274900EBC00001EB800517463046C4
:10A4C000FFF786FF30B1204600F044F820B111209C
:10A4D000BDE8F0871020FBE76F61AE604FF4907726
:10A4E0004FF0000839462068FFF71AFE4FF4AC76AB
:10A4F00031462068FFF714FE2068AA686969C0F831
:10A500004425C0F8481520684FF00109C0F80890AC
:10A510006868D0B9BA4651462068FFF7FCFD074687
:10A5200031462068FFF7F7FD0743F4D010B14FF034
:10A530000F0808E02068C0F80C9031462068FFF74B
:10A54000EAFD0028F9D0002068614046C0E700001D
:10A55000B0A700200079054900EBC00001EB8000A6
:10A560004069002800D0012070470000B0A70020FB
:10A570002DE9F04105460078002828D115481649F4
:10A580000026401AC008012101EB004710E02869AD
:10A59000805DFCF733FC040009D0112CF7D038465D
:10A5A00022460EA1FFF7CEF92046FCF7A5FB761C4C
:10A5B000A88AB042EBD8A98A2869084410F8010C8F
:10A5C0000D2804D10A20FCF719FC1128FAD0BDE8A7
:10A5D000F081000020BE0200B8BD02004661696C37
:10A5E000656420726563656976696E67204E5553B0
:10A5F000206D6573736167652E204572726F7220DE
:10A60000307825782E20000003490860034801684F
:10A610000029FCD07047000004E5014000E401403F
:10A6200010B528B1032815D10220FDF7A7FA0BE0D9
:10A630000020FDF7A3FA08B1FCF75EFBFDF724FA52
:10A6400008B1FCF759FB33DF002803D0BDE8104008
:10A65000FCF752BB10BDF0B58BB0002601960D463D
:10A6600004468988406901AAFCF730FC0AA8CDE9B4
:10A6700008600227ADF82070ADF822602189A88813
:10A6800008AAADDF002819D1A069002816D00998C2
:10A69000FDF799F9002811D0019E0EB1012030700C
:10A6A000182102A8FBF7FBFE8DF808700394A88818
:10A6B000ADF810000596A16902A888470BB0F0BD5F
:10A6C00070B58D88027900EBC5042273C97BA41D87
:10A6D000012902D0022904D101E0008800E040886D
:10A6E000208021886088814211D92846A5DF012673
:10A6F000B0B1112816D0FFF7F9FC02460B480C49FF
:10A70000401AC00806EB00400AA1FFF71BF9A17927
:10A71000E079814208D92846BDE87040FDF71EBEA9
:10A720006671F4E72671F2E770BD0000B8BD020063
:10A73000B8BD020073645F626C655F6761747463C7
:10A740005F65786368616E67655F6D74755F72657C
:10A75000717565737428292072657475726E6564ED
:10A760002025732E000000007CB506468D88C88821
:10A7700006EBC504A41D172800D2172021888142AA
:10A7800000D8084660800020207121882846B5DF67
:10A7900060B1FFF7ABFC02460F481049401AC008F1
:10A7A000012101EB00400EA1FFF7CCF860790028F1
:10A7B00010D1306900280DD01549D1E90201CDE949
:10A7C0000001ADF802506088ADF8040032696946B6
:10A7D000304690477CBD0000B8BD0200B8BD020005
:10A7E00073645F626C655F67617474735F657863DF
:10A7F00068616E67655F6D74755F7265706C7928EE
:10A80000292072657475726E65642025732E0000B0
:10A8100024B30200F0B587B00C4605468E1D89882A
:10A82000406906AAFCF752FB18216846FBF737FE81
:10A830000195A088069AADF80800039231882B890B
:10A84000002704F11200994202D17389022B0DD026
:10A85000AA8991421ED1A96900291BD08DF80070E8
:10A8600004907089ADF81400A96911E0002A11D094
:10A87000FDF7A9F820B1069901200870022002E036
:10A880000698077003208DF80000A969002901D0FF
:10A890006846884707B0F0BD0068012803D0022849
:10A8A00001D00020704701207047000010B5054915
:10A8B000C20800F00703885C01249C4020438854B0
:10A8C00010BD00007CA700200449084490F9300026
:10A8D000082801DB012070470020704728A70020CE
:10A8E0000449084490F93000082801D2012070473B
:10A8F0000020704728A700202DE9F05F2A4F064668
:10A900004FF0A04A4FF0010B0024381990F9501075
:10A91000491C3CD090F85000314620F0C005284634
:10A92000FEF716FB20B3204600F040F881460AEB04
:10A930008500D0F80007C0F30148B8F1020F18D025
:10A9400002212846FEF7A6FD0BFA05F1CAF82015EC
:10A950002846FDF77DFB57F820204AB14846B9F15B
:10A96000030F11D0B8F1020F05D0B8F1030F07D0D3
:10A970000DE00321E5E74846B9F1010F04D006E0F8
:10A980004846B9F1020F02D1014628469047641C9F
:10A99000042CBAD3324601210020FEF78DFD306829
:10A9A0000028B1D1BDE8F09F28A700200249084443
:10A9B00090F850008009704728A7002010B50C4679
:10A9C000017A052908D0407A38B1084808A1026800
:10A9D0002046FEF73FFC00E01AB106A12046FEF734
:10A9E00039FC2046BDE81040FEF741BC002C002099
:10A9F000257300000D0A000038B5C3880D460446D3
:10AA000033B114A0009015A216A12846FEF722FC2F
:10AA1000217A05291CD0607A48B1A088FEF74CFE47
:10AA2000164951F8202016A12846FEF713FCA088ED
:10AA30000021FFF70DF803461049207A143951F828
:10AA4000202001B02846BDE830400EA1FEF702BC30
:10AA500038BD00001B5B306D000000001B5B313B0C
:10AA600033316D0025734C6F67732064726F7070A3
:10AA70006564202825642925730D0A00002C002018
:10AA8000257300003C25733E2025733A200000000A
:10AA900070B50546FDF7ADFD134C40B1D4E9040295
:10AAA0004FF08071411842F10000C4E90410002108
:10AAB0002846FDF7EBFC30B1606820B1606800F01B
:10AAC0003DFA0020606001212846FDF7DFFC18B147
:10AAD000FDF7BAFEC4E90601284600F081FA2846CF
:10AAE000BDE8704000F034B8782B002070B5054602
:10AAF00000200C460870FDF7A7FED5E90223101AC6
:10AB000063EB010300263146361A994112DAB0F59B
:10AB1000350F03D3FCF714F90B4942184FF4960391
:10AB200000210A48FDF771FD10B10D2806D009E09B
:10AB3000012070BD00210548FDF79EFC284600F06D
:10AB4000FDF92070002070BDFFFFB400802B0020B5
:10AB5000F8B51A4C074600261948FFF78DFAD0B110
:10AB6000616871B1D0E902106268D2E90232C91A93
:10AB7000904120D26068007F18B161681048FFF7EB
:10AB80006AFA00F073F905466946FFF7AFFF98B11E
:10AB9000606840B10AE0606800280CD13846BDE822
:10ABA000F840FDF72EBD3846FDF727FD65609DF89E
:10ABB00000000028D0D1F8BD6660CDE7782B0020DA
:10ABC00060B302000D49022008600020091D0860E2
:10ABD0000A4A4FF40031D83A1160084A0121E03A9C
:10ABE0001160121D1060064AC2F80003034A0548AE
:10ABF0003C321060101D016070470000F07500408D
:10AC000000700040F02A0020074801210160074839
:10AC1000C0F80010D0F80021002AFBD00022C0F8B4
:10AC20000021416070470000007500400070004046
:10AC300038B50021012548B1012810D003280DD1D5
:10AC4000FFF77CFABDE83840FEF7DABA4FF0E020B3
:10AC5000C0F88051BFF34F8FBFF36F8F38BD8DF8B1
:10AC600000106846FCF7F4F8064C207808B9FEF7A7
:10AC7000A7FAE068401CE060A5709DF80000FCF7B2
:10AC80000BF938BD14A700203EB5044609496846B3
:10AC9000FFF7BAF908E000BFD0E90021204690474D
:10ACA00030B16846FFF7C7F902980028F4D13EBDDD
:10ACB00011203EBDF8B402003EB50446084968467E
:10ACC000FFF7A2F907E000BFD0E900212046904736
:10ACD0006846FFF7B0F902980028F5D13EBD0000A4
:10ACE00004B5020002498969002900D0084770476D
:10ACF0007CA600202DE9F0411400884618D00025DC
:10AD00000E4F032608EB050122460020FBF7CEFC80
:10AD10000544241A40B93878002809D008494FF46E
:10AD20007A408847761E05D001203870002CE9D182
:10AD3000BDE8F08100203870FAE70000C42B002045
:10AD4000D1B402002DE9F0410746806A14468846D6
:10AD5000C8B3002531E000BFB96A05EB450001EB3F
:10AD60008006B088801CFE2802D90C20BDE8F08146
:10AD70002288401C08F8020020881622401C80B25D
:10AD8000208008F800202088401C80B2208000EB42
:10AD90000801308800F098F92188084480B22080AA
:10ADA000B28842B1B16871B14044FBF75FFB2088C3
:10ADB000B188084420806D1CEDB297F82C00A842A1
:10ADC000CAD80020D2E7FFE70720CFE70A78062895
:10ADD00022F0FF020A7010D2DFE800F00305070935
:10ADE0000B0D002008E0112006E0212004E03120B6
:10ADF00002E0122000E0222008707047002805D1F0
:10AE00000349012048700020FDF7F2B970470000A7
:10AE100014A7002010B51620FBF7E4FDA0B11148DF
:10AE200090F800044009082811D20121814011F056
:10AE3000EC0F0CD00C4882684FF480016AB10168B5
:10AE400041F48001016010BD42F2010001E042F2D4
:10AE50000200BDE81040FBF74FBF4FF0E020C0F804
:10AE6000001110BD16E000E0B0A800200148FFF777
:10AE700006B9000060B30200C207002A03D000BF79
:10AE80004FF00F0201E04FF0F00201D04FEA011144
:10AE9000044B03EB5003187800EA020040EA01007B
:10AEA0001870704718A800202DE9F84F0746214870
:10AEB0009146884605681E46012269461846FCF7F9
:10AEC00051FFDFF874A060B3009800210446801C95
:10AED0000AE000BF00EA050259F821C00AEB82022D
:10AEE000401C491CC2F80CC0B142F3D34FEA1749C9
:10AEF000FDF7B8FA611C29400AEB810149EA0042DA
:10AF00002C40CA600AEB8401C86867F3C50066F389
:10AF1000891068F39F2020F00300401C20F00400FB
:10AF2000C8609AF8000001E0FEF7ECFB0028FBD1B6
:10AF3000BDE8F88FD02B002054AA002070B504463D
:10AF4000124800250078F8B1F4B1207FE0B1FDF798
:10AF50007BFCD4E90223801A994110D32069002692
:10AF600000B92677D4E905108847206960B1217FB0
:10AF700051B1D4E9022110187141C4E902012146FE
:10AF80000348FFF768F80125284670BD782B00209C
:10AF900060B302000F49002008600F480121C16022
:10AFA0000C4B06220C331A600A4A121D1160094B21
:10AFB0000A223C331A600A04C0F80423074BC0225B
:10AFC00083F800244FF0E0230215C3F8002101604C
:10AFD0007047000004A5004000A000400AE000E027
:10AFE000F8B51B4C69462068FDF702FF00260127D3
:10AFF000184D29E0017821B101290CD002291BD17B
:10B0000014E041680A7FBAB90F77416810480830E8
:10B01000FFF721F810E041686868814201D16E6055
:10B020000AE00B480830FFF731F805E0FFF71EFF94
:10B0300008B10677FAE72F7069462068FDF7CDFE64
:10B0400069462068FDF7D4FE0028D3D1F8BD000082
:10B0500058B30200782B0020F8B50B4C0D4606467D
:10B0600069462068FDF7AEFE58B106704560694636
:10B070002068FDF7C8FE10B10448FDF7A7FA0020CC
:10B08000F8BD0420F8BD000058B30200802B00205A
:10B09000034880684108034800224068FBF790BEDF
:10B0A000602B002050B3020070B50C4605464FF4EB
:10B0B0008E71FFF72AF8216AA068415C206A401C63
:10B0C0002062C5F81C1570BD0870000A4870022087
:10B0D000704700002DE9F05F8346DDE90A4A994692
:10B0E00090460D460846012703E000BFB0FBF8F08C
:10B0F0007F1C4045FAD2B94500D94F465FEACA7075
:10B1000012D18CB15FEA8A7002D5B9F1000F01D07B
:10B11000202607E0302605E031465846641EFCF73D
:10B120006BFE0CB1A742F7D35FF00106B9F1010F36
:10B1300002D9A9F1010903E0B5FBF6F0404502D3BD
:10B1400006FB08F6F2E7DFF83C9000BFB5FBF6F02F
:10B1500000FB165519F800105846FCF74DFEB6FBDB
:10B16000F8F6002EF2D15FEACA7009D0002C07D0A1
:10B17000A74205D220215846641EFCF73DFEF5E7A4
:10B18000BDE8F09F76B30200417939B190F82E14F2
:10B1900021B990F8300408B10120704700207047B1
:10B1A00030B40446007A00280AD06088002166DFA7
:10B1B00028B1112802D0616830BC084701202072F4
:10B1C00030BC704770B50C460546FCF74FFE0028B2
:10B1D00007D04268002A04D021462846BDE87040C6
:10B1E000104770BD2DE9FC411646DDE90854CDE954
:10B1F00000541F468046022200F00CF8002807D1B8
:10B20000CDE900543B4610223146404600F002F89A
:10B21000BDE8FC812DE9FC5F0026DDE90C4B994679
:10B2200092468E4680462788354630E0D8F804009E
:10B23000002200EB850069460068019001A864DFE8
:10B24000002830D19DF8000050451FD10EB10021DB
:10B2500000E00221228808441118594522D846B935
:10B26000521C90B2208009F800E02088401C208009
:10B270000126218801A801EB0902694664DF002844
:10B2800011D120889DF80010084420806D1CB8F86A
:10B290000000A842CADC56B12088C01B401E80B204
:10B2A000FF2802D90C20BDE8FC9F09F80700002008
:10B2B000F9E710B5042817D209B1032400E00024EF
:10B2C000FCF786FB4FF0A04101EB8000D0F800179F
:10B2D00021F44031C0F80017D0F8001741EA0441CA
:10B2E000C0F80017002010BD062010BD302C002033
:10B2F000111213140D0E0F10D8A50020F8A5002070
:10B3000028A600200D000300A97A02000E00030009
:10B31000A97A02000F000300A97A020010000300BE
:10B32000A97A0200770A000000000000770A0000F6
:10B33000000000007ADA0000000000009ECADC2451
:10B340000EE5A9E093F3A3B50000406E00000050A5
:10B3500003000000F8A7002028A800200100060034
:10B3600000000000982B0020358202000000000041
:10B370000338FDD8704730313233343536373839F9
:10B380004142434445460000556E6B6E6F776E2018
:10B390006572726F7220636F6465000000000000C8
:10B3A0002CBA020001000000D8B802000200000020
:10B3B000CCB60200030000004CB9020004000000FB
:10B3C000A0B902000500000080B8020006000000DD
:10B3D0001CB802000700000088B902000800000045
:10B3E00094B8020009000000F8B802000A0000004A
:10B3F00014BA02000B000000B4B602000C000000FA
:10B40000ACB802000D0000007CBA02000E00000083
:10B4100078B902000F000000B4B90200100000006B
:10B42000E8B902001100000090BA0200120000000A
:10B4300064BA02001300000000BA0200800000009D
:10B4400034B802008100000070B7020082000000E2
:10B4500030B702008300000010B702008400000033
:10B460004CB702008500000058B8020086000000BA
:10B4700060B9020090000000FCB7020091000000DB
:10B48000F0B6020092000000C0B802000082000086
:10B49000C8B902000182000014B902000282000053
:10B4A00030B90200008400008CB702000184000063
:10B4B00038BA020002840000D4B7020003840000FE
:10B4C000B0B70200D9950200D7950200D1950200CD
:10B4D0000338FDD870470000BCA900207F000000A1
:10B4E0003CAA002000000000000000000000000056
:10B4F0000000000001000007E4B40200F4B4020000
:10B50000080000001CB502002CB502000800000075
:10B510002CB502003CB5020008000000ACBE0200E1
:10B52000B4BE020000000000000000009CBE02004B
:10B53000ACBE0200000000000000000054BE02008B
:10B540005CBE02005CBE02007CBE02007CBE02004B
:10B550008CBE02008CBE020094BE0200D82A0020DD
:10B560003CB502005CB502000800000094BE020079
:10B570009CBE020000000000000000006CB502004C
:10B580007CB50200080000000040404040404040C0
:10B5900040404141414141404040404040404040A6
:10B5A000404040404040404040050202020202024A
:10B5B0000202020202020202022020202020202099
:10B5C00020202002020202020202909090909090AD
:10B5D000101010101010101010101010101010106B
:10B5E00010101010020202020202888888888888DF
:10B5F00008080808080808080808080808080808CB
:10B6000008080808020202024000000089B5020092
:10B6100073645F626C655F6761705F646174615FD2
:10B620006C656E6774685F75706461746528292045
:10B63000287265717565737429206F6E20636F6E53
:10B640006E656374696F6E2030782578207265743A
:10B6500075726E65642025732E00000054686520A5
:10B6600072657175657374656420636F6D62696E70
:10B670006174696F6E206F6620545820616E64207B
:10B680005258207061636B6574206C656E677468D6
:10B690007320697320746F6F206C6F6E67206279FE
:10B6A000202575206D6963726F7365636F6E6473B7
:10B6B0002E0000004E52465F4552524F525F494E97
:10B6C00056414C49445F4441544100004E52465F4C
:10B6D0004552524F525F534F465444455649434595
:10B6E0005F4E4F545F454E41424C454400000000C0
:10B6F0004E52465F4552524F525F46454154555255
:10B70000455F4E4F545F454E41424C45440000005A
:10B710004E52465F4552524F525F4D555445585F09
:10B72000554E4C4F434B5F4641494C454400000049
:10B730004E52465F4552524F525F4D555445585FE9
:10B740004C4F434B5F4641494C4544004E52465F87
:10B750004552524F525F4D555445585F434F4E44EA
:10B760005F494E49545F4641494C45440000000042
:10B770004E52465F4552524F525F4D555445585FA9
:10B78000494E49545F4641494C4544004E52465F3C
:10B790004552524F525F424C455F495053505F52A1
:10B7A000585F504B545F5452554E434154454400EA
:10B7B0004E52465F4552524F525F424C455F495090
:10B7C00053505F504545525F52454A4543544544A6
:10B7D000000000004E52465F4552524F525F424CAD
:10B7E000455F495053505F4C494E4B5F444953436A
:10B7F0004F4E4E4543544544000000004E52465FB4
:10B800004552524F525F4150495F4E4F545F494D30
:10B81000504C454D454E5445440000004E52465F45
:10B820004552524F525F4E4F545F535550504F52F6
:10B83000544544004E52465F4552524F525F4D4F61
:10B8400044554C455F4E4F545F494E495449414C15
:10B85000495A4544000000004E52465F4552524F3F
:10B86000525F4D4F44554C455F414C524541445900
:10B870005F494E495449414C495A45440000000033
:10B880004E52465F4552524F525F4E4F545F464FA5
:10B89000554E44004E52465F4552524F525F494EFC
:10B8A00056414C49445F5354415445004E52465F03
:10B8B0004552524F525F444154415F53495A4500EB
:10B8C0004E52465F4552524F525F494F5F50454E70
:10B8D00044494E47000000004E52465F4552524FC9
:10B8E000525F5356435F48414E444C45525F4D4969
:10B8F0005353494E470000004E52465F4552524F47
:10B90000525F494E56414C49445F4C454E4754485E
:10B91000000000004E52465F4552524F525F445263
:10B92000565F5457495F4552525F414E41434B0069
:10B930004E52465F4552524F525F4452565F5457E3
:10B94000495F4552525F444E41434B004E52465F61
:10B950004552524F525F494E5445524E414C0000A1
:10B960004E52465F4552524F525F53544F524147D9
:10B97000455F46554C4C00004E52465F4552524F73
:10B98000525F4E554C4C00004E52465F4552524F4E
:10B99000525F494E56414C49445F504152414D001F
:10B9A0004E52465F4552524F525F4E4F5F4D454D8E
:10B9B000000000004E52465F4552524F525F464FC4
:10B9C0005242494444454E004E52465F4552524F02
:10B9D000525F4452565F5457495F4552525F4F562B
:10B9E000455252554E0000004E52465F4552524F4E
:10B9F000525F494E56414C49445F41444452000015
:10BA00004E52465F4552524F525F5245534F555228
:10BA1000434553004E52465F4552524F525F494E86
:10BA200056414C49445F464C414753004E52465F95
:10BA300053554343455353004E52465F4552524F70
:10BA4000525F424C455F495053505F4348414E4E10
:10BA5000454C5F414C52454144595F455849535408
:10BA6000530000004E52465F4552524F525F434FC3
:10BA70004E4E5F434F554E54000000004E52465FFD
:10BA80004552524F525F54494D454F5554000000A6
:10BA90004E52465F4552524F525F42555359000035
:10BAA0007761726E696E6700646562756700000099
:10BAB0001B5B313B33306D001B5B306D00000000C1
:10BAC0001B5B313B33316D001B5B313B33326D000F
:10BAD0001B5B313B33336D001B5B313B33346D00FB
:10BAE0001B5B313B33356D001B5B313B33366D00E7
:10BAF0001B5B313B33376D00696E666F00000000E1
:10BB00006572726F7200000073645F626C655F63E0
:10BB100066675F73657428292072657475726E6537
:10BB200064202573207768656E20617474656D707C
:10BB300074696E6720746F2073657420424C455F92
:10BB400047415454535F4346475F53455256494318
:10BB5000455F4348414E4745442E000073645F6291
:10BB60006C655F6366675F7365742829207265740E
:10BB700075726E6564202573207768656E20617428
:10BB800074656D7074696E6720746F2073657420BE
:10BB9000424C455F434F4D4D4F4E5F4346475F56C6
:10BBA000535F555549442E0073645F626C655F6353
:10BBB00066675F73657428292072657475726E6597
:10BBC00064202573207768656E20617474656D70DC
:10BBD00074696E6720746F2073657420424C455FF2
:10BBE00047415454535F4346475F415454525F5456
:10BBF00041425F53495A452E0000000073645F6262
:10BC00006C655F6366675F7365742829207265746D
:10BC100075726E6564202573207768656E20617487
:10BC200074656D7074696E6720746F20736574201D
:10BC3000424C455F434F4E4E5F4346475F4741503E
:10BC40002E00000073645F626C655F6366675F73FC
:10BC5000657428292072657475726E656420257379
:10BC6000207768656E20617474656D7074696E67A5
:10BC700020746F2073657420424C455F4741505FCC
:10BC80004346475F524F4C455F434F554E542E003D
:10BC900073645F626C655F6366675F7365742829B0
:10BCA0002072657475726E656420257320776865EF
:10BCB0006E20617474656D7074696E6720746F2096
:10BCC00073657420424C455F434F4E4E5F43464779
:10BCD0005F474154542E00006E72665F626C655F70
:10BCE0006761747400000000626C655F6E757300BC
:10BCF000636C6F636B000000434C4F434B000000CC
:10BD00004750494F5445000050525300554152543A
:10BD10000000000055415254450000005350494D69
:10BD2000000000006170705F627574746F6E0000D7
:10BD30006170705F74696D65720000007077725F8A
:10BD40006D676D7400000000736F72746C697374BA
:10BD5000000000007274745F6C6F675F6261636BF8
:10BD6000656E6400617070006E72665F7364680077
:10BD70006E72665F7364685F626C65006E72665FA8
:10BD80007364685F736F6300B4BE0200D82A00203A
:10BD900054010000446502000CBF02002C2C00205E
:10BDA000D4A40000D4690200C4B402000000000062
:10BDB00054BD0200C82B0020D8BC020000000303C1
:10BDC000E8BC020000000000F0BC0200000000001F
:10BDD000F8BC02000000000000BD020000000000EE
:10BDE00008BD0200000000000CBD020000000000C1
:10BDF00014BD0200000000001CBD02000000000095
:10BE000024BD02000000000030BD02000000000060
:10BE10003CBD02000000000048BD02000000000020
:10BE200064BD02000000030368BD020000000303BC
:10BE300070BD0200000003037CBD0200000003038C
:10BE4000DC2B0020D42B0020DC2B0020FCA80020C1
:10BE5000180000006577020000000000618F0200FA
:10BE6000C4A50020FB71020090A10020F97502001A
:10BE70000000000069760200000000005179020015
:10BE8000FC2A0020EB90020084A100201D75020016
:10BE900000000000FDAD020000000000C99E02008D
:10BEA00000000000CD9F02000000000031AC020045
:10BEB000000000004154FFFF141201022902131870
:10BEC0002B42201A200812010262040D22100140A8
:10BED00011681220BA400801135AFF04011D13BB58
:10BEE0000214A0BA021AF8041AA8041AB8041AB064
:10BEF000041AC0041AC8041AD0041AD8041AE00498
:0CBF00001AE8041AF00451040090D00369
:040000050002620192
:00000001FF
